:100000000C944F060C9496060C9496060C94960647
:100010000C9496060C9496060C9496060C949606F0
:100020000C9496060C9496060C948F150C949606D8
:100030000C94CF230C9496060C9496060C9496067A
:100040000C9496060C9496060C9496060C949606C0
:100050000C9496060C946F240C9496060C949606B9
:100060000C9496060C9409090C9496060C9496062A
:100070000C9496060C9496060C9496060C94960690
:100080000C9496060C9496060C9496060C94960680
:100090000C9496060C9496060C9496060C94960670
:1000A0000C9496060C9496060C949606320E360E18
:1000B0003A0E3E0E420E460E4A0E4E0E520E560E90
:1000C0005A0E5E0E620E660E6A0E6E0E720E760E80
:1000D0007A0E7E0E820E860E8A0E8E0E920E960E70
:1000E0009A0E9E0EA20EA60EAA0EAE0EB20EB60E60
:1000F000BA0EBE0EFE0E300EC20EC40EC60EC80ED6
:10010000CC0ED00ED40ED80EDD0EE20EE60EEA0EA8
:10011000EE0EF20EF60EFC0EFC0EFC0EFC0EFC0EAD
:10012000FC0EFC0EFC0EFC0EFC0EFC0EFC0EFC0E7F
:10013000FC0EFC0EFC0EFC0EFC0EFC0EFA0E8516E0
:10014000A7169517A7169517EC160F17951764178E
:1001500077177E1A7E1AAB1AAB1A061B421B3A1D82
:100160003A1D5A1B3A1D551C551C101D3A1D3A1DAF
:10017000261D1F141A16041D1B0620211508070929
:10018000190522231C170A0B11801E352B39797B88
:100190007A2C2425180C0E0D1080742A31287C7DB1
:1001A0007F7E26271213330F36802D2E302F3438C2
:1001B0003780253032583A20253038620A000A72DA
:1001C0002F632030313233343536370A00522C3128
:1001D0000D0A0053592C464646340D0A0053482C4C
:1001E000303033430D0A00537E2C360D0A0053572E
:1001F0002C383030300D0A00534D2C340D0A00538A
:10020000532C4B6579626F6172642F4D6F75736506
:100210000D0A00532D2C546D6B42540D0A005346A9
:100220002C310D0A002D2D2D0D0A004578697469B9
:100230006E6720636F6E666967206D6F6465202E40
:100240002E2E0A002B0D0A00760D0A00242424000D
:10025000456E746572696E6720636F6E66696720AC
:100260006D6F6465202E2E2E0A0025630025730D08
:100270000A00522C310D0A0053522C5A0D0A005517
:100280005342206D6F64650A004175746F206D6F75
:1002900064650A00253032750A00253032753A004F
:1002A000253032753A004241543A2025756D560981
:1002B00000757074696D653A2025303275202530DF
:1002C00032753A253032753A253032750A00564279
:1002D00055533A2025580A0052656D6F7465576171
:1002E0006B657570456E61626C65643A2025580ACD
:1002F000000A003F004C4F57004449534348470011
:1003000043484152470046554C4C00626174746545
:1003100072793A20005553422053746174653A2033
:1003200025730A00636F6E6669675F6D6F64653A77
:100330002025580A00726E34325F6175746F636FE6
:100340006E6E656374696E6728293A2025580A0025
:10035000726E34323A2025730A00666F7263655FED
:100360007573623A2025580A0070726F746F636F5C
:100370006C3A2025730A000A2D2D2D2D2D20524E6A
:100380002D343220696E666F202D2D2D2D2D0A0003
:10039000753A20202020202020746F67676C65202C
:1003A000466F72636520555342206D6F64650A0085
:1003B000703A2020202020202070616972696E67C9
:1003C0000A00536C636B3A20202020524E2D3432A9
:1003D00020696E697469616C697A650A0044656CAC
:1003E0003A2020202020656E7465722F657869742C
:1003F00020524E2D343220636F6E666967206D6F18
:1004000064650A00623A2020202020202062617466
:100410007465727920766F6C746167650A00693A59
:1004200020202020202020524E2D343220696E665C
:100430006F0A000A0A2D2D2D2D2D20426C75657432
:100440006F6F746820524E2D34322048656C7020D6
:100450002D2D2D2D2D0A00253032753A253032757F
:100460003A253032750925756D560A004C454420F1
:100470007374617475733A20253032580A00202550
:10048000303258002563005B735D004B6579626F05
:100490006172642073746172740A00524E2D34329A
:1004A00020696E69740A000A55534220696E6974A6
:1004B0000A005B575D005B535D005B525D005B446F
:1004C0005D005B435D001203480048004B004200A2
:1004D00020006D006F00640000000E0374002E0009
:1004E0006D002E006B002E000000040309040902B9
:1004F0007400040100A0320904000001030101009E
:100500000921110100012240000705810308000AAA
:100510000904010001030102000921110100012267
:100520004D000705820308000A09040200010300C8
:10053000000009211101000122360007058303088C
:10054000000A090403000203000000092111010050
:10055000012222000705840320000107050403206F
:1005600000011201100100000008EDFE42420401EA
:10057000010200010631FF0974A101097515002669
:10058000FF009520750881020976150026FF009569
:100590002075089102C005010980A101850216019C
:1005A0000026B7001A01002AB700751095018100D6
:1005B000C0050C0901A1018503160100269C021A41
:1005C00001002A9C02751095018100C005010902F5
:1005D000A1010901A100050919012905150025013D
:1005E00095057501810295017503810105010930A9
:1005F00009311581257F9502750881060938158115
:10060000257F950175088106050C0A38021581259C
:100610007F950175088106C0C005010906A1010585
:100620000719E029E7150025019508750181029554
:1006300001750881010508190129059505750191C4
:10064000029501750391010507190029FF15002680
:10065000FF00950675088100C00A00253032582039
:10066000006B6579626F6172645F7265706F72743E
:100670003A20004C45443A20253032580A004F6E4B
:100680006573686F743A2074696D656F75740A00DC
:10069000290A002575002F002575005D28002564B6
:1006A000002000256400200025640020002564004F
:1006B0007C0025303258006D6F7573656B6579204D
:1006C0005B62746E7C782079207620685D28726584
:1006D000702F61636C293A205B006D6B5F776865F2
:1006E000656C5F74696D655F746F5F6D6178203DE7
:1006F0002025640A006D6B5F776865656C5F6D61CE
:10070000785F7370656564203D2025640A006D6B19
:100710005F74696D655F746F5F6D6178203D202542
:10072000640A006D6B5F6D61785F7370656564204E
:100730003D2025640A006D6B5F696E746572766199
:100740006C203D2025640A006D6B5F64656C6179E7
:10075000203D2025640A006D6B5F776865656C5FDE
:1007600074696D655F746F5F6D6178203D202564ED
:100770000A006D6B5F776865656C5F6D61785F73AC
:1007800070656564203D2025640A006D6B5F7469A7
:100790006D655F746F5F6D6178203D2025640A0090
:1007A0006D6B5F6D61785F7370656564203D2025BA
:1007B000640A006D6B5F696E74657276616C203DD2
:1007C0002025640A006D6B5F64656C6179203D20B3
:1007D00025640A000A00257500363A2077686565A9
:1007E0006C5F74696D655F746F5F6D61783A20004E
:1007F0000A00257500353A20776865656C5F6D6184
:10080000785F73706565643A20000A0025750034CE
:100810003A2074696D655F746F5F6D61783A20008E
:100820000A00257500333A206D61785F7370656545
:10083000643A20000A00257500323A20696E74651A
:100840007276616C286D73293A20000A00257500C4
:10085000313A2064656C6179282A31306D73293A08
:1008600020000A092D2056616C756573202D0A0041
:100870004D3E004D25643E20003F007365742064AA
:10088000656661756C740A00433E20007768657286
:10089000652064656C74613A20637572736F723D94
:1008A00025642C20776865656C3D25640A53656571
:1008B00020687474703A2F2F656E2E77696B69709B
:1008C000656469612E6F72672F77696B692F4D6F51
:1008D0007573655F6B6579730A000A092D204D6F8A
:1008E0007573656B6579202D0A4553432F713A095D
:1008F000717569740A313A0964656C6179282A3125
:10090000306D73290A323A09696E74657276616CCA
:10091000286D73290A333A096D61785F73706565D4
:10092000640A343A0974696D655F746F5F6D61784C
:100930000A353A09776865656C5F6D61785F737039
:100940006565640A363A09776865656C5F74696D38
:10095000655F746F5F6D61780A0A703A0970726939
:100960006E742076616C7565730A643A09736574F8
:100970002064656661756C74730A75703A092B3171
:100980000A646F776E3A092D310A706775703A09FB
:100990002B31300A7067646F776E3A092D31300A57
:1009A0000A7370656564203D2064656C7461202A5B
:1009B000206D61785F7370656564202A20287265F8
:1009C00070656174202F2074696D655F746F5F6D51
:1009D0006178290A003F004D3E2000433E20004C34
:1009E00025640A000A092D20436F6E736F6C652021
:1009F0002D0A4553432F713A09717569740A6D3A8E
:100A0000096D6F7573656B65790A000A092D204DB4
:100A100061676963202D0A643A0964656275670A33
:100A2000783A096465627567206D61747269780A45
:100A30006B3A096465627567206B6579626F6172F4
:100A4000640A6D3A096465627567206D6F75736538
:100A50000A763A0976657273696F6E0A733A09739A
:100A600074617475730A633A09636F6E736F6C65B2
:100A7000206D6F64650A302D343A096C61796572B6
:100A8000302D34284631302D4634290A5061757393
:100A90003A09626F6F746C6F616465720A003F009F
:100AA00074696D65725F72656164333228293A201A
:100AB0002530346C580A006B6579626F6172645F2F
:100AC00069646C653A2025580A006B6579626F612C
:100AD00072645F70726F746F636F6C3A2025580A8E
:100AE00000686F73745F6B6579626F6172645F6CCD
:100AF00065647328293A2025580A000A092D2053D5
:100B00007461747573202D0A004743433A20342ED4
:100B1000392E32204156522D4C4942433A20312E33
:100B2000382E3073766E204156525F415243483A18
:100B300020617672350A004F5054494F4E533A2087
:100B40004C554641204D4F5553454B45592045582E
:100B50005452414B455920434F4E534F4C4520432F
:100B60004F4D4D414E44204B45594D41505F5345EB
:100B70004354494F4E20343039360A004255494CCF
:100B8000443A20366263376261622D646972747917
:100B9000202831333A30363A3431204175672033DA
:100BA000312032303136290A005649443A20307813
:100BB0004645454428742E6D2E6B2E2920504944FD
:100BC0003A203078343234322848484B42206D6F16
:100BD0006429205645523A203078303130340A00AA
:100BE000444553433A20742E6D2E6B2E206B65794D
:100BF000626F617264206669726D776172652066EA
:100C00006F722048484B42206D6F640A000A092D1C
:100C10002056657273696F6E202D0A000A6D6F751C
:100C200073653A206F66660A000A6D6F7573653AE0
:100C3000206F6E0A000A6B6579626F6172643A20F8
:100C40006F66660A000A6B6579626F6172643A20AA
:100C50006F6E0A000A6D61747269783A206F666679
:100C60000A000A6D61747269783A206F6E0A000A90
:100C700064656275673A206F6E0A000A6465627582
:100C8000673A206F66660A000A0A626F6F746C6FBB
:100C9000616465722E2E2E2000433E200000112438
:100CA0001FBECFEFDAE0DEBFCDBF04B603FE27C024
:100CB00080915E0390915F03A0916003B091610306
:100CC0008730904BA740B04BD1F410925E03109246
:100CD0005F03109260031092610314BE84B7877F94
:100CE00084BF0FB6F894A8958091600088618093C6
:100CF0006000109260000FBEE0E0F8E3099511E09B
:100D0000A0E0B1E0E4EFF9E502C005900D92AA3948
:100D1000B107D9F723E0AAE9B1E001C01D92AE35D1
:100D2000B207E1F70E9439100C94F82C0C940000E3
:100D30000FB680959AE0F8947BE27A95F1F708F087
:100D4000589A08F4589886959A95B1F70FBE089569
:100D50000FB680E8F894499BFECF4999FECF96E103
:100D60009A95F1F79CE29A95F1F7869549998068F2
:100D7000C8F70FBE08950FB680E8F89496E19A95EB
:100D8000F1F79CE29A95F1F7869549998068C8F742
:100D900096E19A95F1F7499BFECF0FBE0895FF9318
:100DA000EF93E0919A01F0919B01309709F009953A
:100DB000EF91FF910895FC018591803011F0EFDFF4
:100DC000FBCF0895FF27E0E230E247FF0CC04195DA
:100DD00097FF09C0EDE26095709580959095611D33
:100DE000711D811D911D27FF02C0219530E350E246
:100DF000AA27660F771F881F991FAA1FA41710F034
:100E0000A41B63955A95A9F7AA3008F0A95FA05DC5
:100E1000AF93F395611571058105910541F7ED32A9
:100E200011F4EF93F395F21718F43F93F395FBCF7A
:100E30008F91B5DFFA95E1F70895E991F9918591E0
:100E4000803021F0853219F0AADFF9CF089520E033
:100E5000E89455915532C1F3503311F4689455918B
:100E60005A3348F4505390F3220F022E220F220FD0
:100E7000200D250FF4CF0EF42195899199915336C9
:100E800019F3533729F1533559F1BC0188279927B4
:100E9000E8945C3621F4899199916894559154367F
:100EA00039F446EF7EF077FF0DC08FEF9FEF0AC059
:100EB00055374AE039F0583540E121F0523642E0EA
:100EC00009F00895FF93EF937DDFEF91FF91B7CF86
:100ED000FF93EF93FC0181918030B9F360DFFBCF8A
:100EE000FF93EF9368DFF1CFDF93CF93CDB7DEB7FA
:100EF0002596A3DFCF91DF91089514B88FEF85B9C0
:100F0000549A5C9808958FEF84B980E485B9549A17
:100F10005C9A8FE19EE40197F1F700C0000008950C
:100F20008FEF84B980E485B957985F9A2E9A2F98ED
:100F30000E947D07E4EAF1E088E08E0F11928E13A3
:100F4000FDCFECE9F1E088E08E0F11928E13FDCF1A
:100F500084EA91E09093AF018093AE018CE991E037
:100F60009093AD018093AC0108950F931F93CF939D
:100F7000DF938091AC019091AD012091AE01309151
:100F8000AF013093AD012093AC019093AF018093FA
:100F9000AE015C9B0E948307C0E0D0E001E010E05E
:100FA00080E090E025B1207C2C2BAC0133E0440F95
:100FB000551F3A95E1F7242B25B9EAE1EA95F1F7B7
:100FC00000C0E091AC01F091AD01EC0FFD1F20815C
:100FD00030E0082E02C0359527950A94E2F720FDEF
:100FE0002F9AF5E3FA95F1F70000E6B52E982AE17D
:100FF0002A95F1F700C04091AE015091AF01DA019E
:10100000AC0FBD1F4F9B0AC09801082E01C0220FD4
:101010000A94EAF720953C91232308C06C9198012B
:10102000082E01C0220F0A94EAF7262B2C9326B52E
:101030006E2F70E02E1718F026B530E004C026B5EC
:1010400030E021503F4F261B370B2630310558F03A
:10105000E091AC01F091AD01EC0FFD1F2081FA0190
:10106000EC0FFD1F20833AE13A95F1F700C02F986D
:101070002E9AEBE2F1E03197F1F700C00000019603
:101080008830910509F08ECFA091AE01B091AF01EB
:10109000AC0FBD1FE091AC01F091AD01EC0FFD1F55
:1010A0009C918081981751F00E940D246093B001AB
:1010B0007093B1018093B2019093B3012196C8302F
:1010C000D10509F06DCF5C9B1BC080915503853025
:1010D00021F080915503811113C06091B00170918E
:1010E000B1018091B2019091B3010E94432461311A
:1010F00077428105910520F00E947D070E94902390
:1011000081E0DF91CF911F910F9108952091AE0161
:101110003091AF01F901E80FF11D808108950F931F
:101120001F93CF93DF938EEB91E00E94DB06C0E02C
:10113000D0E002EB11E0E091AE01F091AF01EC0FD5
:10114000FD1F80810E9466231F928F93DF93CF93B0
:101150001F930F930E94740721960F900F900F908A
:101160000F900F900F90C830D10529F7DF91CF91E4
:101170001F910F9108950C9483070C947D07569A44
:1011800081FF02C05E9A08955E98089588E080937A
:10119000CC001092CD00E9ECF0E080818069808382
:1011A000808188608083EAECF0E080818083EBECD2
:1011B000F0E080818083559A5D98789408959091AD
:1011C000B5012091B4019217D1F030E0F901EA5451
:1011D000FE4F80812F5F3F4F33272093B401492F6B
:1011E00050E0921718F4241B350B03C0241B350B59
:1011F0003395233031050CF05D9890E008958FEF22
:101200009FEF08959091C80095FFFCCF8093CE008A
:1012100008951F920F920FB60F9211242F933F93B0
:101220004F935F938F939F93EF93FF938091B501BB
:1012300090E0AC014F5F5F4F2091B401241741F063
:101240003091CE00FC01EA54FE4F30834093B5014B
:101250003091B501822F90E0432F50E0841B950B15
:10126000321708F0939503970CF45D9AFF91EF9174
:101270009F918F915F914F913F912F910F900FBE52
:101280000F901F9018958091CE0208950895809137
:10129000CE0208950895089508950895CF93DF9399
:1012A0008D3C9105B9F1B8F4853B9105A9F148F45D
:1012B000833B9105D1F1843B9105D1F5D0E0C0E2AB
:1012C0003BC0873B910571F150F18C3C910581F554
:1012D000D0E0C8E031C08A3E9105C1F040F4823EC2
:1012E0009105B1F0893E910519F5D0E124C0813214
:1012F00022E0920749F0833222E09207D9F08A383F
:101300009140B1F4D2E017C0D4E015C0D0E213C0D0
:10131000D0E411C0D0E80FC0D0E0C1E00DC0D0E0F3
:10132000C2E00AC0D0E0C4E007C0D0E0C0E104C021
:10133000D0E001C0D1E0C0E08DEF0E94020983E05F
:101340000E94020983E00E9402098D2F0E94020977
:101350008C2FDF91CF910C940209CF93DF93EC0196
:101360008DEF0E94020985E00E94020982E00E943E
:10137000020988810E94020989810E9402098A81EA
:101380000E9402098B81DF91CF910C940209CF93C7
:10139000DF93EC018DEF0E94020989E00E940209AF
:1013A00081E00E94020988810E94020980E00E9477
:1013B00002098A810E9402098B810E9402098C81A4
:1013C0000E9402098D810E9402098E810E940209F9
:1013D0008F81DF91CF910C9402090C94DF08EF927A
:1013E000FF920F931F93CF938C010E9401247C01E5
:1013F000C0E0C7010E9419248017910798F40E9449
:10140000DF089C012F3F8FEF380751F02D3041F05E
:101410002A3041F0EC2FF0E0EA54FD4F2083CF5FFB
:10142000C73138F3EC2FF0E0EA54FD4F108286EB21
:1014300092E0CF911F910F91FF90EF9008950C943F
:10144000020981B3881F8827881F0895879A8F9A79
:10145000089585B7806885BF85B7806885BF0E947D
:10146000260A86988E9A81988998559A5D980C9448
:10147000C608879A8F9808958FB1869581700895D0
:101480008FB186FB882780F908958093CE02089556
:10149000CF93DF93CAE6D2E00E94ED098F3F2FEF92
:1014A000920759F09F938F93DF93CF930E94740715
:1014B0000F900F900F900F90EFCFDF91CF91089585
:1014C000CF93DF93FC018491EF012196882321F0D3
:1014D0000E941F0AFE01F7CF2FEF89E698E1215005
:1014E00080409040E1F700C0000084E690E00E9458
:1014F000EF098093CF029093D0029F938F938DE654
:1015000092E09F938F930E9474070E94480A0F9065
:101510000F900F900F908091CF029091D002DF91A9
:10152000CF9108950E94CD179093150180931401D7
:101530000E945B1D80E091E00E94C8170E94390A5A
:101540000E94400A8111FCCF80E592E00E94DB06F8
:101550002FEF85EB95E3215080409040E1F700C0EC
:1015600000008CE492E00E94600AEFEFFBE42DE1C2
:10157000E150F0402040E1F700C000000E94480A1E
:1015800088E492E00E94600AFC018081863721F0A5
:1015900084E492E00C94600A08958BE292E00E9449
:1015A000DB0685E292E00E94600A0E94260A0E9401
:1015B0005B1D80911401909115010C94C8170C9437
:1015C000750F8F929F92AF92BF92CF92DF92EF9260
:1015D000FF920F931F93CF93DF9392E0B92E0EE704
:1015E00014E024E8E22E24E0F22EAA24A39433E0AF
:1015F000932E4CE6C42E44E0D42E0E94ED09EC015B
:10160000019609F441C08091D3028130F9F028F0AD
:10161000823009F1833021F134C0CE3FD10519F475
:10162000A092D302EACFC038D10528F4DF93CF933C
:10163000FF92EF9204C0DF93CF931F930F930E940A
:1016400074070F900F900F900F90D7CF2297C9F487
:10165000B092D302D2CF2197A1F49092D302CDCFF2
:101660008091400380FF0AC0DF93CF93DF92CF9237
:101670000E9474070F900F900F900F908C2F0E9474
:10168000450A1092D302B9CF8091D502811121C0B1
:101690008091D40281111DC00E943C0A81110AC0B0
:1016A0000E94CD178A50914029F00E945B1D8AE06C
:1016B00091E00DC00E943C0A882359F00E94CD178A
:1016C0008651914031F00E945B1D86E191E00E94BD
:1016D000C8178091D1029091D2020E941924893EAC
:1016E00023E0920708F461C028EE33E0B9010E94BC
:1016F000A82C629FC001639F900D729F900D1124D2
:101700002091D1023091D202820F931F9093D20286
:101710008093D1020E941310833011F481E001C044
:1017200080E00E94640F0E940D2428EE33E040E028
:1017300050E00E94D02C49015A018CE3C82ED12CD4
:10174000E12CF12CCA01B901A70196010E94D02C0D
:10175000672B682B692B49F50E94DC0F2091400311
:1017600020FF23C09F938F931F921F92C501B40146
:1017700020E13EE040E050E00E94D02CC22FA701C3
:1017800096010E94D02C3F932F931F92CF9387E511
:1017900094E09F938F930E9474078DB79EB70A962B
:1017A0000FB6F8949EBF0FBE8DBF0E943C0A8111F8
:1017B00007C00E94400A882319F06E9A769802C0EA
:1017C0006E9A769ADF91CF911F910F91FF90EF90D3
:1017D000DF90CF90BF90AF909F908F9008958F92A1
:1017E0009F92AF92BF92CF92DF92EF92FF921F93A0
:1017F000CF93DF9300D000D0CDB7DEB7833109F4AB
:101800008CC008F05BC08B3009F466C08C3009F4E2
:101810008FC0853009F0FBC10E940D2428EE33E013
:1018200040E050E00E94D02C49015A010E94DC0F98
:101830009F938F9386EA92E09F938F930E94740701
:10184000C501B40120E13EE040E050E00E94D02C10
:101850005F934F933F932F9320EA32E03F932F9370
:1018600069837A838B839C830E9474078CE3C82EE0
:10187000D12CE12CF12C69817A818B819C81A7018B
:1018800096010E94D02C5F934F933F932F938AE948
:1018900092E09F938F930E947407C501B401A70142
:1018A00096010E94D02C9F938F937F936F9384E92E
:1018B00092E09F938F930E94740740C1883361F038
:1018C00020F4883109F440C1A2C1873409F46DC104
:1018D0008C3409F456C19BC183E394E00E94DB067B
:1018E0008EE194E00E94DB0684E094E00E94DB0637
:1018F0008DED93E00E94DB0682EC93E00E94DB0614
:1019000080EB93E00E94DB061091D50211117DC19E
:1019100080E993E00E94DB067EC10E94920A88E77C
:1019200092E00E94600A82E792E00E94600A6BC126
:1019300087E793E00E94DB060E94CD178A50914012
:1019400019F08FE291E002C089E291E09F938F93BA
:1019500089E693E09F938F930E9474078091D4024D
:101960001F928F938AE593E09F938F930E94740751
:101970000E943C0A0FB6F894DEBF0FBECDBF8111A6
:1019800007C00E94400A811106C088E391E005C0AB
:1019900084E391E002C08BE391E09F938F9380E515
:1019A00093E09F938F930E9474070E94210A1F92D5
:1019B0008F9385E393E09F938F930E9474078091A8
:1019C000D5021F928F9384E293E09F938F930E949E
:1019D0007407809155030FB6F894DEBF0FBECDBFDC
:1019E0008823B9F0809155038130B1F0809155037F
:1019F0008230A9F0809155038330A1F08091550386
:101A0000843099F080915503853091F080E791E022
:101A100011C088E491E00EC080E491E00BC083E542
:101A200091E008C08BE591E005C085E691E002C039
:101A300082E791E09F938F9385E193E09F938F934B
:101A40000E9474078BE093E09F938F930E9474072A
:101A50000E9413100F900F900F900F900F900F9007
:101A6000813059F038F0823059F0833061F485EFDD
:101A700092E00BC086E093E008C080E093E005C0F0
:101A800089EF92E002C083EF92E09F938F930E94D0
:101A900074070F900F9081EF92E09F938F930E94B5
:101AA0007407809153031F928F9388ED92E09F9368
:101AB0008F930E9474078091D90081701F928F9339
:101AC0008EEC92E09F938F930E9474070E940D24E6
:101AD00028EE33E040E050E00E94D02C69017A010A
:101AE0009CE3892E912CA12CB12CCA01B901A5012E
:101AF00094010E94D02C7F936F93C701B60120E11F
:101B00003EE040E050E00E94D02C122FA50194014D
:101B10000E94D02C3F932F931F921F93C701B601B1
:101B200020E831E541E050E00E94D02C3F932F9314
:101B300081EB92E09F938F930E9474070FB6F89405
:101B4000DEBF0FBECDBF61C08091D502811162C0E2
:101B50001091D402112339F089E892E00E94DB064B
:101B60001092D40258C08FE792E00E94DB0681E019
:101B70008093D4020E945B1D86E191E00E94C81709
:101B800044C00E94210A182F882341F00E94920A23
:101B900081E0809350038093D5023DC00E94CD0A1E
:101BA000109250031092D50230C08091D50281115D
:101BB00002C00E94920A8EE192E00E94600A83E1D4
:101BC00092E00E94600A8FEF91E00E94600A88EF25
:101BD00091E00E94600A8EEE91E00E94600A87EE1A
:101BE00091E00E94600A8DED91E00E94600A83ED11
:101BF00091E00E94600A8DEC91E00E94600A809161
:101C0000D502811102C00E94CD0A11E004C01091DA
:101C1000D50201C010E0812F0F900F900F900F9010
:101C2000DF91CF911F91FF90EF90DF90CF90BF9009
:101C3000AF909F908F900895CF93C82F0E94C52298
:101C4000827291E009F490E04C2F50E0FA01349751
:101C5000E934F10508F0D0C0EA5AFF4F0C94F22C99
:101C60008BE12DC19111CCC081E629C19111CAC06F
:101C700082E625C19111C8C083E621C19111C6C079
:101C800084E61DC19111C4C085E619C19111C2C07D
:101C900086E615C19111C0C087E611C19111BEC081
:101CA00088E60DC19111BCC089E609C19111BAC085
:101CB0008AE605C19111B8C08BE601C19111B6C089
:101CC0008CE6FDC09111B4C08DE6F9C09111B2C08F
:101CD0008EE6F5C09111B0C08FE6F1C09111AEC093
:101CE00080E7EDC09111ACC081E7E9C09111AAC0B5
:101CF00082E7E5C09111A8C083E7E1C09111A6C0B9
:101D000084E7DDC09111A4C085E7D9C09111A2C0BC
:101D100086E7D5C09111A0C087E7D1C091119EC0C0
:101D200088E7CDC091119CC089E7C9C091119AC0C4
:101D30008AE7C5C0911198C081E3C1C0911196C0D6
:101D400082E3BDC0911194C083E3B9C0911192C0E8
:101D500084E3B5C0911190C085E3B1C091118EC0EC
:101D600086E3ADC091118CC087E3A9C091118AC0F0
:101D700088E3A5C0911188C089E3A1C0911186C0F4
:101D800080E39DC088E09BC089E099C080E297C055
:101D900091117EC08DE293C091117CC08DE38FC004
:101DA00091117AC08BE58BC0911178C08DE587C009
:101DB000992309F475C08CE782C0992309F472C095
:101DC0008CE77DC0911170C08BE379C091116EC01A
:101DD00087E275C091116CC080E671C091116AC034
:101DE0008CE26DC0911168C08EE269C0911166C02D
:101DF0008FE265C080E063C080E261C08AE05FC0BE
:101E000081E45DC082E45BC083E459C084E457C0D0
:101E100085E455C086E453C087E451C088E44FC0D0
:101E200089E44DC08AE44BC08BE449C08CE447C0D0
:101E30008DE445C08EE443C08FE441C080E53FC0DF
:101E400081E53DC082E53BC083E539C084E537C00C
:101E500085E535C086E533C087E531C088E52FC00C
:101E600089E52DC08AE52BC081E229C080E427C026
:101E700083E225C084E223C085E221C08EE51FC035
:101E800086E21DC08AE21BC088E219C089E217C041
:101E90008FE515C08BE213C08BE711C08DE70FC033
:101EA0008CE50DC08CE50BC08AE309C082E207C057
:101EB0008EE705C08CE303C08EE301C08FE30E9470
:101EC0001F0A81E0CF910895833019F4859A7D9A95
:101ED0000895813011F4859A06C0823019F4859AEC
:101EE0008D9A089585988D98089581E00E94640FD9
:101EF0002FEF89E698E1215080409040E1F700C043
:101F0000000082E00E94640F2FEF89E698E12150E3
:101F100080409040E1F700C0000081E00E94640F23
:101F20002FEF89E698E1215080409040E1F700C012
:101F3000000082E00E94640F2FEF89E698E12150B3
:101F400080409040E1F700C0000080E00E94640FF4
:101F500080EC80937C0087E080937A0081E9809315
:101F60007E0081E080937F008BE380937D00849AE4
:101F70008C9808958091D90080FF1CC090B331B334
:101F800085988D9AEFE9FFE03197F1F700C00000E6
:101F90008FB185FB882780F920B390722F7D292B84
:101FA00020BB91B3232F20729F7D922B91BB91E098
:101FB0008927089580E00895CF93DF9300D0CDB7AF
:101FC000DEB7849A8C9A80917A00806880937A0038
:101FD0008FE99FE00197F1F700C0000080917A003F
:101FE000806480937A0080917A0086FDFCCF809196
:101FF0007800909179009A83898380917A008F7715
:1020000080937A00849A8C9829813A8145E0429F96
:10201000C001439F900D1124805591090F900F909E
:10202000DF91CF9108958091D90080FD0C94BA0F73
:102030000E94DC0F8C3A2DE0920720F481E080931F
:10204000D60205C085379E4010F01092D6028091CE
:10205000D602811102C082E0089583E00895CF93F3
:10206000C82F0E9498068C2F0E94C01080E0CF914C
:102070000895CF9384B7877F84BF0FB6F894A8954F
:1020800080916000886180936000109260000FBEB4
:1020900090E080E80FB6F89480936100909361001F
:1020A0000FBE0E9414150E9471158091E200846099
:1020B0008093E2008FE290E10E946123509A589A47
:1020C0005198599A7894CFEF80915503843051F00C
:1020D0008FE79EE30197F1F700C000000E94AD1763
:1020E000C15091F787EA94E00E94DB060E94290A1A
:1020F0000E94DF0A8BE994E00E94DB060E945E18D2
:102100000E943C0A811103C08AE091E002C086E18E
:1021100091E00E94C8178BE894E00E94DB060E94C1
:102120003C0A882319F1809155038530F9F487E83A
:1021300094E00E94DB060E94BD080E9490230E944A
:1021400090230E9490230E9490230E9490230E943B
:1021500090230E94902380915303882301F30E94CF
:10216000B9238823E1F20E946713D9CF0E94621835
:102170000E94AD170E94E10AD2CF8091E202089539
:102180009FB7F8941092D9029FBF90915503943055
:1021900009F057C09091E9009F703091EC00232F17
:1021A000217030FD20E8922B24E02093E90020915B
:1021B000EB0020FF43C02091EE0027FF3FC020919D
:1021C000D702222321F02091E80025FF37C010928A
:1021D000D70226E03091E80035FD15C03091550357
:1021E000343061F53091EB0035FD28C0215021F4E9
:1021F00081E08093D70222C0EFE9FFE03197F1F749
:1022000000C00000E7CF8093F1008091E80085FDD9
:102210000AC08091E80080FFFCCF8091E8008E77B3
:102220008093E80006C08FB7F89421E02093D9028C
:102230008FBF9F709093E90080E008959F70909306
:10224000E9008FEF0895CF93DF9300D01F92CDB7B1
:10225000DEB79C0180915503843019F593E0998392
:102260003B832A839093E9008FEF9091E80081509F
:1022700095FD06C095ED9A95F1F700008111F5CF17
:102280008091E80085FF0DC040E050E063E070E021
:10229000CE0101960E947D138091E8008E77809395
:1022A000E8000F900F900F90DF91CF910895CF939A
:1022B000DF9300D01F92CDB7DEB7209155032430B5
:1022C00021F522E029839B838A8383E08093E900C0
:1022D0008FEF9091E800815095FD06C095ED9A959D
:1022E000F1F700008111F5CF8091E80085FF0DC066
:1022F00040E050E063E070E0CE0101960E947D1363
:102300008091E8008E778093E8000F900F900F90F7
:10231000DF91CF910895209155032430F1F422E00C
:102320002093E9002FEF3091E800215035FD06C0E1
:1023300035ED3A95F1F700002111F5CF2091E80035
:1023400025FF0BC040E050E065E070E00E947D1387
:102350008091E8008E778093E8000895CF93DF9313
:1023600020915503243039F521E02093E9002FEF27
:102370003091E800215035FD06C035ED3A95F1F772
:1023800000002111F5CF2091E80025FF14C0EC01D9
:1023900040E050E068E070E00E947D138091E8002A
:1023A0008E778093E80088E0FE01AAEDB2E001900C
:1023B0000D928A95E1F7DF91CF91089582EC94E038
:1023C0000E94DB0680915403811109C00E941415FC
:1023D0000E9471158091E20084608093E20008956C
:1023E0008EEB94E00E94DB061092540308958AEB72
:1023F00094E00C94DB062091D8022F5F822F62E3D9
:102400000E949C2C992319F02093D80208951092D1
:10241000D8028091D902882371F1809155038430CC
:1024200041F58091E9008F702091EC00922F91701E
:1024300020FD90E8892B94E09093E9009091EB00C7
:1024400090FF14C09091EE0097FF10C09091E800AB
:1024500095FF03C01092F100F9CF9091E80090FF32
:1024600005C09091E8009E779093E8008F7080936C
:10247000E9001092D902089542E061EC81E00E94E7
:102480008E1442E061EC82E00E948E1442E061EC26
:1024900083E00E948E1442E261EC84E00C948E147E
:1024A00080915703833009F453C030F4813071F0C8
:1024B000823009F48CC008958A3009F478C08B30DA
:1024C00009F45EC0893009F09AC020C0809156039B
:1024D000813A09F094C08091E800877F8093E800FA
:1024E00080915A0390915B03892B21F468E08AED77
:1024F00092E003C060E080E090E070E00E94CA13C8
:102500008091E8008B778093E800089580915603CE
:10251000813209F074C080915A0390915B03892B3A
:1025200009F06DC08091E800877F8093E80080917A
:10253000E80082FD05C0809155038111F8CF5FC08E
:102540008091F1008093E2028091E8008B7753C084
:1025500080915603813A09F052C080915A039091BC
:102560005B03892B09F04BC08091E800877F809343
:10257000E8008091E80080FFFCCF8091200136C008
:10258000809156038132D9F580915A0390915B0373
:10259000892BA9F58091E800877F8093E8000E944D
:1025A000C31480915803809320010C945B1D80918B
:1025B0005603813221F58091E800877F8093E800FF
:1025C0000E94C314809159038093E302089580917F
:1025D0005603813AA1F48091E800877F8093E80058
:1025E0008091E80080FFFCCF8091E3028093F100AE
:1025F0008091E8008E778093E8000C94C3140895CE
:10260000089586EB94E00E94DB060C9400130C9472
:10261000CD2382EB94E00E94DB060C940713292F54
:10262000332723303105C9F064F42130310581F0BE
:102630002230310509F043C084E790E02EEE34E00B
:1026400042C021323105F1F02232310541F137C06B
:1026500082E190E022E635E036C09927813091058D
:1026600041F08230910541F0892B49F5EAEEF4E022
:1026700005C0EAEDF4E002C0E6ECF4E0849190E0FD
:102680009F0121C06430D8F4E62FF0E0EE0FFF1F69
:10269000E857FE4F2081318189E090E014C064301A
:1026A00070F470E0FB01EE0FFF1FE058FE4F208139
:1026B0003181FB01E458FE4F808190E004C080E04E
:1026C00090E020E030E0FA0131832083089580E13A
:1026D00089BD82E189BD09B400FEFDCF8091D8009B
:1026E0008F7D8093D8008091E00082608093E0002D
:1026F0008091E00081FDFCCF0895CF92DF92EF92B0
:10270000FF920F931F93CF93DF93EC018B017A011C
:102710000E94E214811135C0E114F10439F0F7018F
:1027200080819181081B190BC80FD91FC12CD12C96
:102730000115110529F18091E80085FD18C08091EF
:10274000E8008E778093E8000E94AD17E114F10451
:1027500049F0F70180819181C80ED91ED182C082D3
:1027600085E00FC00E94E214882311F30AC089910A
:102770008093F10001501109FFEFCF1ADF0AD8CF83
:1027800080E0DF91CF911F910F91FF90EF90DF904C
:10279000CF90089520915C0330915D032617370791
:1027A00048F06115710539F42091E8002E772093E7
:1027B000E80001C0B90140E061157105A9F120915F
:1027C0005503222309F443C0253009F442C0209167
:1027D000E80023FD40C02091E80022FD32C0209196
:1027E000E80020FFE9CF4091F3002091F20030E0B3
:1027F000342BFC01CF016115710559F028303105EA
:1028000040F481918093F100615071092F5F3F4F37
:10281000F1CF41E02830310509F040E02091E80097
:102820002E772093E800C8CF4111C9CF0AC080910C
:102830005503882361F0853061F08091E80083FDC5
:102840000AC08091E80082FFF2CF80E0089582E024
:10285000089583E0089581E0089520915C0330910C
:102860005D032617370748F06115710539F420918B
:10287000E8002E772093E80001C0B901FC0120E0B8
:102880006115710591F180915503882309F440C0C9
:10289000853009F43FC08091E80083FD3DC0809100
:1028A000E80082FD2FC08091E80080FFE9CF2091F1
:1028B000F3008091F20090E0922B6115710559F0C0
:1028C0008830910540F424912093F10031966150B5
:1028D00071090196F2CF21E0089709F020E080917C
:1028E000E8008E778093E800CBCF2111CCCF0AC0CF
:1028F00080915503882361F0853061F08091E80074
:1029000083FD0AC08091E80082FFF2CF80E0089545
:1029100082E0089583E0089581E00895982F97302C
:1029200058F59093E900981739F07091EC002091D8
:10293000ED005091F00003C0242F762F50E021FFCE
:1029400019C03091EB003E7F3093EB003091ED00E9
:102950003D7F3093ED003091EB0031603093EB0020
:102960007093EC002093ED005093F0002091EE0066
:1029700027FF07C09F5FD3CF8F708093E90081E06E
:10298000089580E008958091560387FF11C08091DB
:10299000E80082FD05C0809155038111F8CF11C078
:1029A0008091E8008B770BC080915503882349F014
:1029B0008091E80080FFF8CF8091E8008E778093C7
:1029C000E80008952091E4003091E50095E64091FB
:1029D000EC00842F817040FF22C08091E80080FDD0
:1029E0001CC080915503882391F0853091F080912F
:1029F000EB0085FD10C04091E4005091E5004217C6
:102A0000530729F39A01915011F784E0089582E069
:102A1000089583E0089581E0089580E0089540914D
:102A2000E80042FFDECF08950E9482150E948A15B9
:102A3000E0EEF0E0808181608083E8EDF0E080816D
:102A40008F77808319BCA7EDB0E08C918E7F8C933B
:102A500080818F7E80831092540308950F931F937B
:102A6000CF93DF930E9482150E948A15C8EDD0E0B3
:102A700088818F77888388818068888388818F7D2B
:102A8000888319BC1092550310925103109253037E
:102A90001092520300EE10E0F80180818B7F80835A
:102AA00088818160888342E060E080E00E948E142B
:102AB000E1EEF0E080818E7F8083E2EEF0E08081C5
:102AC00081608083808188608083F80180818E7F2F
:102AD0008083888180618883DF91CF911F910F91DE
:102AE0000895E8EDF0E080818F7E8083E7EDF0E0EF
:102AF00080818160808384E082BF81E08093540381
:102B00000C942E15E8EDF0E080818E7F808310928A
:102B1000E20008951092DA001092E10008951F92E9
:102B20000F920FB60F9211242F933F934F935F9301
:102B30006F937F938F939F93AF93BF93EF93FF9385
:102B40008091E10082FF0BC08091E20082FF07C00C
:102B50008091E1008B7F8093E1000E94FB118091C6
:102B6000DA0080FF1FC08091D80080FF1BC08091D9
:102B7000DA008E7F8093DA008091D90080FF0DC04B
:102B800080E189BD82E189BD09B400FEFDCF81E00D
:102B9000809355030E94DE1105C019BC10925503A5
:102BA0000E94F0118091E10080FF19C08091E20045
:102BB00080FF15C08091E2008E7F8093E2008091BB
:102BC000E20080618093E2008091D800806280936F
:102BD000D80019BC85E0809355030E9401138091B1
:102BE000E10084FF30C08091E20084FF2CC080E1CE
:102BF00089BD82E189BD09B400FEFDCF8091D80076
:102C00008F7D8093D8008091E1008F7E8093E100DA
:102C10008091E2008F7E8093E2008091E2008160EB
:102C20008093E20080915103882311F084E007C073
:102C30008091E30087FD02C081E001C083E08093C2
:102C400055030E9409138091E10083FF24C0809105
:102C5000E20083FF20C08091E100877F8093E10044
:102C600082E080935503109251038091E1008E7FA2
:102C70008093E1008091E2008E7F8093E20080915A
:102C8000E20080618093E20042E060E080E00E9428
:102C90008E140E94F711FF91EF91BF91AF919F9118
:102CA0008F917F916F915F914F913F912F910F90F5
:102CB0000FBE0F901F9018951F93CF93DF93CDB742
:102CC000DEB7AA970FB6F894DEBF0FBECDBFE6E51C
:102CD000F3E088E08E0F9091F10091938E13FBCF7B
:102CE0000E9450128091E80083FF1FC1809156031B
:102CF00090915703492F50E04A30510508F015C113
:102D0000FA01E156FF4F0C94F22C803881F08238A2
:102D100009F00BC180915A038F708093E900809174
:102D2000EB0085FB882780F91092E90006C08091AE
:102D3000520390915303911182609091E800977F24
:102D40009093E8008093F1001092F100C8C0282F02
:102D50002D7F09F0EAC0882319F0823061F0E5C0C8
:102D600080915803813009F0E0C0933009F080E091
:102D7000809353032BC080915803811127C0809109
:102D80005A038F7009F4D1C08093E9002091EB00C1
:102D900020FF1CC0933021F48091EB00806214C0AE
:102DA0009091EB0090619093EB0021E030E0A9015D
:102DB00002C0440F551F8A95E2F74093EA00109233
:102DC000EA008091EB0088608093EB001092E900AC
:102DD0008091E800877F86C08111A7C010915803B9
:102DE0001F778091E3008078812B8093E3008091AE
:102DF000E800877F8093E8000E94C3148091E80078
:102E000080FFFCCF8091E30080688093E300111184
:102E100002C082E001C083E08093550386C08058E1
:102E2000823008F082C080915803909159038C3D04
:102E300053E0950779F583E08A838AE289834FB767
:102E4000F894DE01139620E03EE051E2E32FF0E03B
:102E500050935700E49120FF03C0E295EF703F5F6D
:102E6000EF708E2F90E0EA3010F0C79601C0C09648
:102E70008D939D932F5F243149F74FBF8091E800D8
:102E8000877F8093E8006AE270E0CE0101960E949D
:102E9000CA1314C0AE014F5F5F4F60915A030E9486
:102EA0000F13BC01892B09F440C09091E800977F73
:102EB0009093E80089819A810E942D148091E80006
:102EC0008B778093E80031C0803879F58091E800F5
:102ED000877F8093E800809151038093F100809177
:102EE000E8008E778093E8000E94C3141EC0811111
:102EF0001CC0909158039230C0F48091E800877F05
:102F00008093E800909351030E94C3148091510371
:102F1000811106C08091E30087FD02C081E001C0FD
:102F200084E0809355030E943C128091E80083FF67
:102F30000AC08091E800877F8093E8008091EB00D1
:102F400080628093EB00AA960FB6F894DEBF0FBEA6
:102F5000CDBFDF91CF911F910895CF9380915503FD
:102F60008823A1F0C091E900CF709091EC00892FE7
:102F7000817090FD80E8C82B1092E9008091E800F4
:102F800083FD0E945C16CF70C093E900CF91089535
:102F90009093E9028093E80208958091E80290916D
:102FA000E9020895E091E802F091E902309721F0FA
:102FB0000190F081E02D099480E00895EF92FF9256
:102FC0000F931F93CF93DF93E091E802F091E90212
:102FD0003097B1F18C010280F381E02D0995809149
:102FE000400382FF2DC080FF04C081E696E00E946E
:102FF000DB06E80118E08BE5E82E86E0F82E8091EC
:10300000400380FF0BC088811F928F93FF92EF9245
:103010000E9474070F900F900F900F9011502196FF
:103020001111EDCF8091400380FF0AC089E596E041
:10303000DF91CF911F910F91FF90EF900C94DB06E1
:10304000DF91CF911F910F91FF90EF900895E09144
:10305000E802F091E902309721F00480F581E02D3B
:10306000099408952091E6023091E70282179307B0
:1030700071F09093E7028093E602E091E802F0910C
:10308000E902309721F00680F781E02D0994089538
:103090002091E4023091E5028217930771F090933A
:1030A000E5028093E402E091E802F091E9023097B2
:1030B00021F00084F185E02D099408950E94F82301
:1030C0000C949007CF92DF92EF92FF920F931F9391
:1030D000CF93DF9300D000D000D0CDB7DEB70E94F1
:1030E000B5078BEEC82E82E0D82E00E010E0E02E6F
:1030F000802F0E948608F60141916F01F42EF82678
:10310000B1F40F5F1F4F0830110589F78FEF8983E6
:103110008A831B820E9401248160782F9D838C8387
:1031200049815A816B818D810E94211947C09091FC
:10313000400391FF04C08E830E948F088E8120E09F
:1031400030E04F2D50E0922FBA01022E02C075954B
:1031500067950A94E2F760FF2BC02983EA8221E099
:1031600030E0690102C0CC0CDD1C9A95E2F790E0DA
:103170008C219D21892B09F420E02B830E940124BE
:103180008160782F9D838C8349815A816B818D81E9
:103190000E94211949815A816B817C818D810E9415
:1031A0007D23F801E551FD4F8081C826C08206C00D
:1031B0002F5F3F4F2830310531F6A3CF0E947C238B
:1031C0000E94F0261091EA020E94D217181741F1CE
:1031D0000E94D2178093EA029091400392FF0EC0A2
:1031E00090FF0CC01F928F9383E796E09F938F937D
:1031F0000E9474070F900F900F900F908091EA0239
:1032000026960FB6F894DEBF0FBECDBFDF91CF91EB
:103210001F910F91FF90EF90DF90CF900C948E2331
:1032200026960FB6F894DEBF0FBECDBFDF91CF91CB
:103230001F910F91FF90EF90DF90CF9008950C9425
:10324000BF08CF93DF93CDB7DEB72B970FB6F894B7
:10325000DEBF0FBECDBF942F4F83252F58876987C0
:103260007A878B874A855B85452B21F02F3F09F5AF
:103270009F3FF9F4DE01119686E0FD0111928A95D7
:10328000E9F785E0FE01379601900D928A95E1F706
:1032900049815A816B817C818D819E810E94FE1FB4
:1032A0002B960FB6F894DEBF0FBECDBFDF91CF9146
:1032B00008954F81588569857A858B850E947D2385
:1032C000D9CFCF93882309F4A4C0C82F8CEF8C0FDB
:1032D000813A48F48C2F0E94162A81119AC08C2FB3
:1032E0000E9489220CC080E28C0F883058F4C7708D
:1032F00081E001C0880FCA95EAF70E94C822CF91E9
:103300000C940C238BE58C0F833078F4C53A29F0AC
:10331000C63A31F083E890E005C081E890E002C051
:1033200082E890E0CF910C94321888E58C0F8531BB
:1033300008F06FC0C83A61F1C93A69F1CA3A71F14F
:10334000CB3A79F1CC3A81F1CD3A89F1CE3A91F18B
:10335000CF3A99F1C13BA1F1C03BA9F1C23BB1F118
:10336000C33BB9F1C43BC1F1C53BC9F1C63BD1F187
:10337000C73BD9F1C83BE1F1C93BE9F1CA3BF1F1E7
:10338000CB3BF9F1CC3B09F43FC080E090E03EC07C
:1033900082EE90E03BC089EE90E038C08AEE90E08B
:1033A00035C085EB90E032C086EB90E02FC083EB18
:1033B00090E02CC084EB90E029C087EB90E026C021
:1033C0008CEC90E023C08DEC90E020C083E891E08D
:1033D0001DC08AE891E01AC082E991E017C084E933
:1033E00091E014C081E292E011C083E292E00EC04D
:1033F00084E292E00BC085E292E008C086E292E0AF
:1034000005C087E292E002C08AE292E0CF910C947C
:103410004818CF910895882329F19CEF980F913A8D
:1034200018F40E94A6220DC090E2980F983058F42C
:10343000877091E001C0990F8A95EAF7892F0E9461
:10344000CE220C940C239BE5980F933020F480E05F
:1034500090E00C943218885A853120F480E090E096
:103460000C9448180895882321F00E94C8220C94D7
:103470000C230895882321F00E94CE220C940C2363
:103480000895CF92DF92EF92FF920F931F93CF9305
:10349000DF9300D000D000D0CDB7DEB725E0FC012F
:1034A000DE01119601900D922A95E1F7FC01408111
:1034B0003181F280258122952F7063817481672B81
:1034C00009F4D8C23F3F19F44F3F09F4D3C26C014D
:1034D00049833A8389819A812E830E944822182F3A
:1034E000092F0E9447220E945721E02FE295EF709A
:1034F000F0E0E755FF4F2E810C94F22C802F807F57
:10350000902F9F70092F882311F00295007FFF20D4
:1035100049F0002309F45FC2802F0E94DB220E9441
:103520000C2359C2812F0E940B1A002309F4A2C256
:10353000802F0E94E12226960FB6F894DEBF0FBEC0
:10354000CDBFDF91CF911F910F91FF90EF90DF9052
:10355000CF900C940C23802F807F902F9F70092F89
:10356000803211F00295007F112319F0113001F122
:1035700029C0FF20A9F0802F222349F1213039F5FD
:1035800026960FB6F894DEBF0FBECDBFDF91CF9168
:103590001F910F91FF90EF90DF90CF900C94EB2252
:1035A000222319F0213009F465C20E94F4222CC0B4
:1035B000FF20E9F0263008F05DC20E94C52280237A
:1035C00029F022C0FF20F1F0211115C0802F26968E
:1035D0000FB6F894DEBF0FBECDBFDF91CF911F9124
:1035E0000F91FF90EF90DF90CF900C94331A25301D
:1035F00008F040C209C0F601858180FFECC18F70E0
:103600008583E4CF2111FBC1802F69C1202F26952E
:103610002695237030E02115310521F02130310548
:10362000C9F028C2FF2021F0812F902F937002C093
:1036300080E090E026960FB6F894DEBF0FBECDBFB7
:10364000DF91CF911F910F91FF90EF90DF90CF907E
:103650000C943218FF2021F0812F902F937002C01C
:1036600080E090E026960FB6F894DEBF0FBECDBF87
:10367000DF91CF911F910F91FF90EF90DF90CF904E
:103680000C944818812FFF2019F00E94762502C063
:103690000E94DE2526960FB6F894DEBF0FBECDBF82
:1036A000DF91CF911F910F91FF90EF90DF90CF901E
:1036B0000C946326802F837009F078C0F110DAC172
:1036C000812F829586958770880F880F912F9F7024
:1036D000C92ED12CE12CF12C082E04C0CC0CDD1C01
:1036E000EE1CFF1C0A94D2F714FF12C04FE050E00A
:1036F00060E070E004C0440F551F661F771F8A9575
:10370000D2F7CB01BA01609570958095909503C072
:1037100060E070E0CB01202F269526952370422F84
:1037200050E042305105D1F04330510559F16C2938
:103730007D298E299F294130510541F126960FB6EA
:10374000F894DEBF0FBECDBFDF91CF911F910F91D7
:10375000FF90EF90DF90CF900C946C216C297D2925
:103760008E299F2926960FB6F894DEBF0FBECDBFD7
:10377000DF91CF911F910F91FF90EF90DF90CF904D
:103780000C947E210E946C21C701B60126960FB6CB
:10379000F894DEBF0FBECDBFDF91CF911F910F9187
:1037A000FF90EF90DF90CF900C945A21FF2019F0FA
:1037B000802F817001C08695882309F45BC1812F19
:1037C000829586958770880F880F912F9F70C92EDC
:1037D000D12CE12CF12C082E04C0CC0CDD1CEE1CED
:1037E000FF1C0A94D2F714FF12C04FE050E060E0D3
:1037F00070E004C0440F551F661F771F8A95D2F7EB
:10380000CB01BA01609570958095909503C060E0FA
:1038100070E0CB01202F269526952370422F50E093
:1038200042305105D1F04330510559F16C297D29C1
:103830008E299F294130510541F126960FB6F89403
:10384000DEBF0FBECDBFDF91CF911F910F91FF90D3
:10385000EF90DF90CF900C9423226C297D298E2944
:103860009F2926960FB6F894DEBF0FBECDBFDF911D
:10387000CF911F910F91FF90EF90DF90CF900C941C
:1038800035220E942322C701B60126960FB6F8946E
:10389000DEBF0FBECDBFDF91CF911F910F91FF9083
:1038A000EF90DF90CF900C941122103F41F118F46B
:1038B000103E48F48BC0123F09F450C0D8F1133FBA
:1038C00009F460C083C01F70802F8F71FF2021F02A
:1038D0000E94AA21812F7BCE0E94CB21812F269688
:1038E0000FB6F894DEBF0FBECDBFDF91CF911F9111
:1038F0000F91FF90EF90DF90CF900C943A1AFF2039
:10390000A9F0253008F0B6C0802F8F7126960FB62B
:10391000F894DEBF0FBECDBFDF91CF911F910F9105
:10392000FF90EF90DF90CF900C94F021263008F0BC
:10393000A1C0EACFFF20A1F0802F8F7126960FB68D
:10394000F894DEBF0FBECDBFDF91CF911F910F91D5
:10395000FF90EF90DF90CF900C94AA21FF2061F3AD
:10396000802F8F7126960FB6F894DEBF0FBECDBFA5
:10397000DF91CF911F910F91FF90EF90DF90CF904B
:103980000C94CB21FF2091F0802F8F7126960FB6DB
:10399000F894DEBF0FBECDBFDF91CF911F910F9185
:1039A000FF90EF90DF90CF900C94952126960FB664
:1039B000F894DEBF0FBECDBFDF91CF911F910F9165
:1039C000FF90EF90DF90CF900C949021FF20A1F01A
:1039D000222309F4B1CF812F26960FB6F894DEBFCB
:1039E0000FBECDBFDF91CF911F910F91FF90EF9050
:1039F000DF90CF900C946119222309F4B1CF812F6D
:103A000026960FB6F894DEBF0FBECDBFDF91CF91E3
:103A10001F910F91FF90EF90DF90CF900C940B1AB5
:103A2000402F4F70612FC6010E94F02426960FB6DA
:103A3000F894DEBF0FBECDBFDF91CF911F910F91E4
:103A4000FF90EF90DF90CF900C94A220402F4F700A
:103A5000612FC60126960FB6F894DEBF0FBECDBF0C
:103A6000DF91CF911F910F91FF90EF90DF90CF905A
:103A70000C94F32426960FB6F894DEBF0FBECDBF8C
:103A8000DF91CF911F910F91FF90EF90DF90CF903A
:103A900008950E94E8220E94B7220E940C230E94EF
:103AA00095270E94632680E090E00E94321880E013
:103AB00090E00C9448180E94D8220C94491D0E9452
:103AC0004822292F22952F7030E02C3031054CF4FC
:103AD0002A3031056CF4225031092230310588F446
:103AE00007C02C30310549F02F30310531F009C0C5
:103AF000803E48F0803F29F406C093FB882780F978
:103B0000089580E0089581E00895CF93DF9300D079
:103B100000D01F92CDB7DEB70F900F900F900F908F
:103B20000F90DF91CF910895CF93DF9300D000D015
:103B300000D0CDB7DEB726960FB6F894DEBF0FBE25
:103B4000CDBFDF91CF9108951F93CF93DF93C091A5
:103B5000F30216E08091F402C81799F0D0E01C9FA0
:103B6000F0011D9FF00D1124EB50FD4F408151815C
:103B700062817381848195810E94941D2196C77012
:103B8000E9CFDF91CF911F91089540912503509186
:103B90002603609127037091280380912903909157
:103BA0002A030C94941D80912A0382958F7009F04A
:103BB00054C080912703882309F44FC08091F302F9
:103BC000A091F4026091250370912603409128038F
:103BD00050912903B6E08A1709F43FC090E04115DF
:103BE0005105C1F17F3F11F46F3FA1F1B89FF00182
:103BF000B99FF00D1124EB50FD4F218172132AC0A3
:103C00002081621327C02281211124C023813481A5
:103C10002417350710F421503109241B350B2C32A1
:103C20003140C0F420912A032F70206120932A0391
:103C300026E0289FF001299FF00D1124E650FD4F4A
:103C400080818F708061808385E293E00E94411AB9
:103C50000C94A41D01968770BECF0895CF92DF9279
:103C6000EF92FF920F931F93CF93DF93CDB7DEB701
:103C700062970FB6F894DEBF0FBECDBF8C0185E012
:103C8000F801DE011D9601900D928A95E1F7D801A9
:103C90004C9111965C91119712966C911297139614
:103CA000CD90DC901497309125037091260380917C
:103CB000280390912903009709F473C17F3F19F4F9
:103CC0003F3F09F46EC1E0902703EE2009F4C5C020
:103CD00020912A03C816D90650F0F601E81BF90B0B
:103CE000CF01FF24F3948C329140C8F009C0809535
:103CF00090958C0D9D1DFF24F3948C32914078F0AB
:103D0000F12C207F09F0C6C07C2DD98AC88A898908
:103D10000E94851D85E293E00E94411AB1C0822F66
:103D2000807F09F045C0751313C0341311C06111B1
:103D30000FC02F70206120932A030E94C51D85E2C9
:103D400093E00E94411A80912A03F80185832EC0D6
:103D5000CD2819F15F3F11F44F3FF9F0F62E6111B4
:103D60001CC08091F3022091F40236E0821709F41E
:103D70005BC090E0389FF001399FF00D1124EB50AB
:103D8000FD4F7181571306C07081471303C07281C4
:103D9000711103C001968770E9CFF62E662309F4EE
:103DA0001DC180912A03816080932A03F12C16C1E2
:103DB000751309C0341307C0611105C080912A032F
:103DC000F8018583C8C04D875E878D859E856A8B87
:103DD0000E945F1D6A898823E1F16623D1F1209159
:103DE0002A03822F82958F7090E0029774F0809161
:103DF00025039091260398878F831986DB86CA86D0
:103E00002C87CE0107960E94411A86E0F801A5E2B0
:103E1000B3E001900D928A95E1F70E94D31D0E94B4
:103E2000C51DFF24F394DAC04D875E878D859E857E
:103E30000E944822292F22952F7030E02230310530
:103E40000CF0BFC09F7009F0B9C0805E883008F4E4
:103E5000C5C0C8010E94411AE4CFC816D90608F4AB
:103E600053C0F601E81BF90BCF018C32914008F4E6
:103E700053C0F12C7C2DD98AC88A89890E94851D5E
:103E8000E5E2F3E086E0DF011D928A95E9F70E9402
:103E9000C51DA4C0751314C0341312C0611110C025
:103EA00080912A03F8018583C8010E94411A86E0A7
:103EB000E5E2F3E0DF011D928A95E9F7FE2C8EC062
:103EC0004D875E878D859E856A8B0E945F1D6A89FE
:103ED000882309F4BECF662309F4BBCF20912A03BF
:103EE000822F82958F7090E002970CF48ECF809194
:103EF0002503909126039A8389831B82DD82CC82DD
:103F00002E83CE0101967FCF809590958C0D9D1DBF
:103F10008C32914008F0ADCFF62E662309F499CF8C
:103F200075132EC034132CC020912A0320FD1FC00E
:103F3000822F82958F70D9F0D80115962C93159702
:103F40008F3049F08F5F982F9295907F822F8F70DE
:103F5000892B15968C93C8010E94411A86E0F801BE
:103F6000A5E2B3E001900D928A95E1F790CF86E04B
:103F7000F801A5E2B3E001900D928A95E1F72EC019
:103F80004D875E878D859E850E945F1D81113DCF87
:103F900080912A03816080932A03C8010E94411AFC
:103FA0001DC0662309F455CF4D875E878D859E859C
:103FB0000E945F1D882309F44CCF27CF811145CF84
:103FC0000DC0243031050CF044CF9F7009F43DCF73
:103FD000D80115969C91907F09F037CF8F2D62966E
:103FE0000FB6F894DEBF0FBECDBFDF91CF911F910A
:103FF0000F91FF90EF90DF90CF9008951F93CF9394
:10400000DF93CDB7DEB72C970FB6F894DEBF0FBEA7
:10401000CDBF4F83588769877A878B879C87CE016E
:1040200007960E942E1E882369F08F8198852A8525
:104030003B85232BF1F19F3F09F063C08F3F09F0CF
:1040400060C037C086E0FE013796DE011196019010
:104050000D928A95E1F76F817885EA85FB85309727
:1040600041F17F3F11F46F3F21F12091F40230E0E4
:10407000C9010196877099274091F30250E0841797
:10408000950709F447C069837A83FD83EC8396E042
:10409000929FD001939FB00D1124AB50BD4FFE01F4
:1040A000319601900D929A95E1F78093F4020E9467
:1040B000A41D16E08091F3029091F4028917C1F1DA
:1040C000189FC00111248B509D4F0E942E1E8823E3
:1040D00079F1E091F3021E9FF0011124EB50FD4FA6
:1040E0004081518162817381848195810E94941DF8
:1040F0008091F30290E00196877099278093F302F4
:10410000D9CF4F81588569857A858B859C850E949A
:10411000941DCFCF0E945B1D1092F4021092F30207
:10412000E5E2F3E086E0DF011D928A95E9F7C1CF71
:104130002C960FB6F894DEBF0FBECDBFDF91CF91A6
:104140001F910895DF92EF92FF920F931F93CF93E9
:10415000DF93FC01892B09F48AC0E12CF12CDD24CA
:10416000D394EF0121968491853709F461C058F406
:10417000843708F04EC0843008F06AC08130D1F036
:10418000823071F174C0883709F45DC050F486370D
:1041900009F455C0873709F06AC08E2D0E94D522D8
:1041A00054C09CE7980F903708F061C08F770E9449
:1041B0000B1A50C08F010E5F1F4FFE01849190E2D9
:1041C000980F983050F48770FD2D01C0FF0F8A952D
:1041D000EAF78F2F0E94DB2214C00E94611913C0DE
:1041E0008F010E5F1F4FFE01C49180E28C0F88305B
:1041F00060F4C7708D2D01C0880FCA95EAF70E9440
:10420000E1220E940C23E80125C08C2F0E940B1A8A
:10421000FACF9F012E5F3F4FFE01C491CC2369F07E
:104220008FE99FE00197F1F700C00000C150F6CF81
:104230009F012E5F3F4FFE01F490E9010BC00E94E9
:10424000C522E82E07C00E94D8220E940C2302C07B
:104250000E9461198F2D882341F0EFE9FFE031972B
:10426000F1F700C000008150F6CFFE017ACFDF9158
:10427000CF911F910F91FF90EF90DF900895609381
:104280002F037093300380933103909332030E9485
:104290008C230C94491D60932B0370932C03809303
:1042A0002D0390932E030E948D230C94491D089595
:1042B0000C943F210F931F9300912F031091300313
:1042C0002091310330913203602B712B822B932B81
:1042D0001F910F910C943F210F931F9300912F0377
:1042E0001091300320913103309132036023712308
:1042F000822393231F910F910C943F210F931F93BF
:1043000000912F031091300320913103309132033B
:1043100060277127822793271F910F910C943F21CB
:1043200060E070E0CB010C944B210F931F9341E0B0
:1043300050E060E070E08A019B0104C0000F111F93
:10434000221F331F8A95D2F7C901B8011F910F911F
:104350000C944B210F931F9341E050E060E070E01C
:1043600004C0440F551F661F771F8A95D2F78091AE
:104370002B0390912C03A0912D03B0912E038A0161
:104380009B01082B192B2A2B3B2BC901B8011F912C
:104390000F910C944B210F931F9341E050E060E08C
:1043A00070E004C0440F551F661F771F8A95D2F72F
:1043B000409550956095709580912B0390912C03BA
:1043C000A0912D03B0912E038A019B01082319238C
:1043D0002A233B23C901B8011F910F910C944B2153
:1043E0000F931F9341E050E060E070E004C0440F81
:1043F000551F661F771F8A95D2F780912B039091E6
:104400002C03A0912D03B0912E038A019B01082754
:1044100019272A273B27C901B8011F910F910C9436
:104420004B210F931F9300912B0310912C0320918C
:104430002D0330912E03602B712B822B932B1F9118
:104440000F910C944B210F931F9300912B0310910C
:104450002C0320912D0330912E036023712382239E
:1044600093231F910F910C944B210F931F93009155
:104470002B0310912C0320912D0330912E036027E4
:104480007127822793271F910F910C944B21089538
:10449000CF92DF92EF92FF920F931F93CF93DF9310
:1044A0008C01C0902F03D0903003E0903103F09046
:1044B000320340912B0350912C0360912D03709196
:1044C0002E03C42AD52AE62AF72ACFE1D0E0D70165
:1044D000C6010C2E04C0B695A795979587950A94AA
:1044E000D2F780FF07C0B8018C2F0E94C52481300D
:1044F000910531F4219758F7B80180E00E94C52456
:10450000DF91CF911F910F91FF90EF90DF90CF90AF
:1045100008952091210130912201F90132969FEFF7
:1045200040E05191581789F09F3F19F4511101C093
:10453000942F4F5F4630A9F79F3F39F0F901E90FFB
:10454000F11D97FDFA958283089508952091210128
:1045500030912201F9013296285F3F4F90819813E4
:1045600001C010823196E217F307C1F7089581E088
:1045700090E0E0912101F0912201E80FF91F1082F3
:10458000019688309105A9F7089580913F03089519
:1045900090913F03892B80933F03089580959091DC
:1045A0003F03892380933F03089580933F03089539
:1045B00010923F03089590913E03892B80933E0310
:1045C0000895809590913E03892380933E0308953A
:1045D00010923E030895809335030E940124909326
:1045E00034038093330308951092350310923403FB
:1045F0001092330308958091210190912201FC01D2
:1046000031969C01285F3F4F80E0919191118F5F1F
:10461000E217F307D1F70895E0912101F09122010B
:1046200080913F038083E0912101F09122019081EC
:1046300080913E03892B8083809135038823D9F1B3
:104640000E94012420913303309134038217930791
:1046500048F00E9401242091330330913403821BDF
:10466000930B0AC00E94012420913303309134033C
:1046700020953095820F931F8C32914070F080917D
:10468000400380FF08C08EE796E09F938F930E94BF
:1046900074070F900F900E94F422E0912101F09195
:1046A0002201908180913503892B80830E94FB2217
:1046B00081110E94F42280912101909122010C9499
:1046C000DE1790939B0180939A0108958295982F0D
:1046D0009C7C392F36953695282F237344E0249FF0
:1046E000C0011124932F982B292F2A7A2695892FE0
:1046F0008575880F822B08950895CF93DF9300D09E
:1047000000D01F92CDB7DEB70F900F900F900F9093
:104710000F90DF91CF910895089508950C941F197B
:1047200080915503843021F11092410320E488E107
:1047300090E00FB6F894A895809360000FBE209388
:10474000600083B7817F846083BF83B7816083BF4C
:104750007894889583B78E7F83BF0FB6F894A89519
:1047600080916000886180936000109260000FBEAD
:104770000895CF930E94BB080E94B5070E94BD0810
:10478000C0E08C2F0E948608811104C0CF5FC83022
:10479000C1F701C081E0CF9108950C945B1D1F9279
:1047A0000F920FB60F9211248F939F93AF93BF93E5
:1047B00080914103811113C0809142039091430382
:1047C000A0914403B09145034196A11DB11D809372
:1047D000420390934303A0934403B0934503BF91D6
:1047E000AF919F918F910F900FBE0F901F901895D2
:1047F00082E084BD93E095BD9AEF97BD80936E00F3
:1048000008952FB7F8948091420390914303A091AB
:104810004403B09145032FBF08952FB7F8946091DA
:1048200042037091430380914403909145032FBF4D
:104830000895CF92DF92EF92FF920F931F932FB7BD
:10484000F894409142035091430360914403709166
:1048500045032FBF6A017B01EE24FF248C0120E079
:1048600030E0C016D106E206F30610F441505109BB
:104870009A01281B390BC9011F910F91FF90EF90EE
:10488000DF90CF900895CF92DF92EF92FF920F9337
:104890001F932FB7F894C0904203D0904303E09049
:1048A0004403F09045032FBF97018601061B170BA9
:1048B000280B390BC616D706E806F90618F0C90109
:1048C000B80106C0C901B801615071098109910997
:1048D0001F910F91FF90EF90DF90CF9008951F925E
:1048E0000F920FB60F9211248F939F93AF93BF93A4
:1048F0008091420390914303A0914403B0914503FA
:104900000196A11DB11D8093420390934303A09390
:104910004403B0934503BF91AF919F918F910F9046
:104920000FBE0F901F9018950E941415F8942FEF4A
:1049300087EA91E6215080409040E1F700C00000F6
:1049400087E090EBDC0180935E0390935F03A0937C
:104950006003B09361039CE088E10FB6F894A895DA
:10496000809360000FBE90936000FFCF28E0929F7D
:10497000F0011124E80FF11DEE58FE4F8491982F9D
:1049800090778F7092959F700895CF93C82FCB0129
:104990000E94B624292F30E0E82FF0E0A90164E05E
:1049A000440F551F6A95E1F74E2B5F2B4038510598
:1049B00019F480E090E012C088E0C89F200D311DFE
:1049C000112484E0220F331F8A95E1F7E20FF31FD1
:1049D000EE0FFF1FE050F84985919491CF91089513
:1049E00080E090E0089508958091480380FF0BC017
:1049F0006091260185E0689FB00111247595679547
:104A0000759567952BC081FF09C06091260185E0EF
:104A1000689FB00111247595679520C082FF07C07B
:104A20006091260185E0689FB001112417C0909124
:104A300049039923D1F060912501961788F72091B9
:104A4000260185E0289F90011124929FA001939F49
:104A5000500D112470E0CA010E94BC2C6038710511
:104A600040F46115710539F002C065E070E0862FF1
:104A700008958FE7089581E008958091480380FFAD
:104A800008C06091240170E07595679575956795EC
:104A900021C081FF06C06091240170E07595679583
:104AA00019C082FF04C06091240170E010C0909191
:104AB00049039923C1F0609123019617A0F78091D3
:104AC0002401899FC001112470E00E94BC2C603831
:104AD000710528F46115710521F0862F08958FE77F
:104AE000089581E0089561E070E0F4CF803F21F403
:104AF0000E94F424819504C0813F29F40E94F4248B
:104B000080934C030895823F21F40E94F424819500
:104B100004C0833F29F40E94F42480934B0308953A
:104B2000893F19F40E943D2505C08A3F31F40E9457
:104B30003D25819580934D0308958B3F21F40E947C
:104B40003D25819504C08C3F29F40E943D2580932A
:104B50004E030895843F21F480914A03816017C079
:104B6000853F21F480914A03826011C0863F21F481
:104B700080914A0384600BC0873F21F480914A03EF
:104B8000886005C0883F31F480914A03806180933A
:104B90004A0308958D3F21F48091480381600BC042
:104BA0008E3F21F480914803826005C08F3F29F435
:104BB000809148038460809348030895803F39F4CE
:104BC00080914C0387FF6CC010924C0369C0813FF9
:104BD00029F480914C031816BCF362C090914B03EA
:104BE000823F29F497FF5CC010924B0359C0833F6A
:104BF00019F41916CCF354C0893F41F480914D0348
:104C000018160CF04DC010924D034AC08A3F29F48B
:104C100080914D0387FF44C0F6CF8B3F39F48091DC
:104C20004E0387FF3DC010924E033AC08C3F29F4DB
:104C300080914E031816BCF333C0843F21F4809159
:104C40004A038E7F17C0853F21F480914A038D7FF0
:104C500011C0863F21F480914A038B7F0BC0873FB0
:104C600021F480914A03877F05C0883F31F4809109
:104C70004A038F7E80934A0313C08D3F21F48091B5
:104C800048038E7F0BC08E3F21F4809148038D7FB7
:104C900005C08F3F29F4809148038B7F80934803A0
:104CA00080914B0381110EC080914C0381110AC089
:104CB00080914D03811106C080914E03811102C085
:104CC0001092490308958091400383FF7EC087EBD3
:104CD00096E00E94DB0680914A031F928F9382EB3D
:104CE00096E09F938F930E94740780EB96E00E945A
:104CF000DB0680914B03282F082E000C330B3F93CB
:104D00008F938DEA96E09F938F930E9474078BEAAE
:104D100096E00E94DB0680914C03282F082E000CA1
:104D2000330B3F938F9388EA96E09F938F930E9473
:104D3000740786EA96E00E94DB0680914D03282FD7
:104D4000082E000C330B3F938F9383EA96E09F93DA
:104D50008F930E94740781EA96E00E94DB0680919F
:104D60004E03282F082E000C330B3F938F938EE9B0
:104D700096E09F938F930E9474078BE996E00E94C0
:104D8000DB06809149031F928F9388E996E09F93F9
:104D90008F930E94740786E996E00E94DB0680915B
:104DA00048031F928F9383E996E09F938F930E940D
:104DB000740780E996E00E94DB068DB79EB74C969B
:104DC0000FB6F8949EBF0FBE8DBF8AE493E00E9499
:104DD00027180E9401249093470380934603089567
:104DE0001F93CF93DF9380914603909147030E94D6
:104DF0001924AC0190914903992321F020912701B6
:104E000030E006C0209128018AE0289F90011124FB
:104E10004217530708F485C080914B03C0914C039F
:104E2000D0914D0310914E03811107C0C11175C07F
:104E3000D11173C0111171C074C09F3F19F09F5FF1
:104E400090934903181624F40E94F42480934B0392
:104E500080914B0387FF05C00E94F42481958093C5
:104E60004B031C1624F40E94F42480934C0380917D
:104E70004C0387FF05C00E94F424819580934C0366
:104E800060914B03662331F1C0914C03CC2311F1A7
:104E9000062E000C770B880B990B0E94A32B23E3A3
:104EA00033E343E35FE30E94072C0E946B2B609384
:104EB0004B036C2FCC0F770B880B990B0E94A32B05
:104EC00023E333E343E35FE30E94072C0E946B2B51
:104ED00060934C031D1624F40E943D2580934D03DE
:104EE00080914D0387FF05C00E943D2581958093E9
:104EF0004D03111624F40E943D2580934E038091AA
:104F00004E0387FF05C00E943D25819580934E0387
:104F1000DF91CF911F910C9463269F3F09F08FCFB3
:104F200097CFDF91CF911F910895EAE4F3E085E0F8
:104F3000DF011D928A95E9F7109249031092480308
:104F400008958AED98E00E94DB061F9281E08F931E
:104F50001F9285E08F938CE898E09F938F930E9437
:104F600074070F900F900F900F900F900F9008956F
:104F70008330E9F128F4813061F0823009F108953D
:104F8000853009F462C008F449C0863009F474C061
:104F9000089580912801262F30E0280F311D2F3FE2
:104FA000310524F4680F6093280103C08FEF8093CC
:104FB0002801809128011F928F9385EC97E072C0A1
:104FC00080912701262F30E0280F311D2F3F31051A
:104FD00024F4680F6093270103C08FEF80932701AB
:104FE000809127011F928F9383EB97E05BC08091A4
:104FF0002601262F30E0280F311D2F3F310524F4E4
:10500000680F6093260103C08FEF80932601809183
:1050100026011F928F9380EA97E044C0809125017A
:10502000262F30E0280F311D2F3F310524F4680F63
:105030006093250103C08FEF8093250180912501A6
:105040001F928F938BE897E02DC080912401262F2B
:1050500030E0280F311D2F3F310524F4680F609395
:10506000240103C08FEF80932401809124011F92BB
:105070008F9382E797E016C080912301262F30E0BE
:10508000280F311D2F3F310524F4680F6093230151
:1050900003C08FEF80932301809123011F928F9390
:1050A00087E597E09F938F930E9474070F900F906E
:1050B0000F900F900895833081F128F4813059F0DA
:1050C0008230D1F00895853009F449C0B8F18630B6
:1050D00009F456C0089580912801681720F4861BB2
:1050E0008093280102C010922801809128011F920C
:1050F0008F9388E497E054C080912701681720F4CB
:10510000861B8093270102C01092270180912701FE
:105110001F928F9386E397E043C080912601681722
:1051200020F4861B8093260102C0109226018091F4
:1051300026011F928F9383E297E032C08091250170
:10514000681720F4861B8093250102C01092250168
:10515000809125011F928F938EE097E021C080916E
:105160002401681720F4861B8093240102C010924A
:105170002401809124011F928F9385EF96E010C047
:1051800080912301681720F4861B8093230102C0BD
:1051900010922301809123011F928F938AED96E054
:1051A0009F938F930E9474070F900F900F900F9012
:1051B0000895CF93C82F1F928F938FED99E09F93FF
:1051C0008F930E94740781E090E0A0E0B0E0BC0102
:1051D000CD0104C0660F771F881F991FCA95D2F7AB
:1051E0000E9458210F900F900F900F90CF910C9428
:1051F0005B1DCF93873288F58E3108F00BC18E305E
:1052000009F487C0D8F4873009F460C08B3009F402
:105210004FC0863009F002C180914003817F8E7FAC
:105220008093400384EE99E00E94DB0689E99CE0CC
:105230000E94DB0681E08093500346C0863109F46A
:10524000B0C020F4803109F47AC0E8C0893109F493
:1052500091C08B3109F449C0E1C0883349F150F461
:10526000893209F4D5C0853309F4D2C0873209F0F8
:10527000D5C0CEC0833409F4CBC028F48A3308F4F7
:10528000CDC08953C8C0883409F0C8C00E945B1DD6
:1052900088E89CE00E94DB062FEF83ED90E321502D
:1052A00080409040E1F700C000000E9494240CC0B0
:1052B0008BE09AE041C08FE69CE00E94DB06809183
:1052C0004003816080934003C1E0ADC08091400302
:1052D000C82FC17080FFEFCF8BE79CE00E94DB06F8
:1052E00080914003817F8E7F3FC09091400391FB6E
:1052F000CC27C0F981E0C827892FC0FB81F98093B2
:105300004003CC2319F082E69CE029C084E59CE0B0
:1053100013C09091400392FBCC27C0F981E0C827CD
:10532000892FC0FB82F980934003CC2319F085E4D8
:105330009CE015C085E39CE00E94DB06C5CF909100
:10534000400393FBCC27C0F981E0C827892FC0FB1D
:1053500083F980934003CC2351F089E29CE00E94C2
:10536000DB06809140038160809340035CC08CE148
:105370009CE0E2CF8DE09CE00E94DB0680EE9BE0AB
:105380000E94DB0689EA9BE00E94DB068CE79BE03B
:105390000E94DB0687E39BE00E94DB0689E09BE03E
:1053A000CBCF8BEF9AE00E94DB060E94D2171F92B0
:1053B0008F9381EE9AE09F938F930E947407809160
:1053C00020011F928F938AEC9AE09F938F930E9403
:1053D00074078091E3021F928F9387EB9AE09F936B
:1053E0008F930E9474070E940D249F938F937F9345
:1053F0006F9380EA9AE09F938F930E9474078DB712
:105400009EB742960FB6F8949EBF0FBE8DBF5CCF7D
:1054100080E001C08D510E94D92856CF8EE99AE0D4
:105420000E94DB06C0E08C2FCF910895CF93C82F48
:1054300080915003813071F020F0823009F44BC02C
:1054400042C1E0912101F09122018081823209F074
:105450003CC107C0E0912101F0912201808182329C
:1054600061F48C2F0E94EF0B811104C08C2F0E94DD
:10547000F9282FC081E090E02CC08C2F0E941C0ED8
:10548000811126C0C431E1F070F4CB3081F0C0311D
:10549000D1F40E94A12787ED99E00E94DB0682E00B
:1054A0008093500315C0C93259F0C83361F484EEBB
:1054B00099E00E94DB068BED99E00E94DB0608C0B4
:1054C0001092500304C185ED99E00E94DB06FFC0F5
:1054D00081E08170FEC0C43228F5CE3108F0C1C031
:1054E000CB30A1F1D0F4C73009F0D3C08EE1809366
:1054F000280182E3809327018AE08093260184E1DA
:105500008093250188E08093240188E28093230121
:105510008BE798E00E94DB06BFC0C33149F1C4317C
:10552000C1F0B7C0CB3409F4A9C028F4C93289F05E
:10553000C83361F0AEC0C13509F49EC0C23509F46C
:1055400099C0CE3409F0A5C06AE09EC00E94A12790
:10555000A3C080914F03882319F010924F039CC081
:1055600088E898E00E94DB0681E080935003B1C098
:1055700082E698E00E94DB0680E598E00E94DB0668
:10558000809128011F928F938DE498E09F938F93D1
:105590000E9474078BE498E00E94DB0689E398E0A0
:1055A0000E94DB06809127011F928F9386E398E08B
:1055B0009F938F930E94740784E398E00E94DB0618
:1055C00085E298E00E94DB06809126011F928F936E
:1055D00082E298E09F938F930E94740780E298E0A4
:1055E0000E94DB068FE098E00E94DB068091250197
:1055F0001F928F938CE098E09F938F930E94740783
:105600008AE098E00E94DB0685EF97E00E94DB06C7
:10561000809124011F928F9382EF97E09F938F9345
:105620000E94740780EF97E00E94DB0689ED97E007
:105630000E94DB06809123011F928F9386ED97E0F5
:105640009F938F930E94740784ED97E00E94DB067E
:105650008DB79EB748960FB6F8949EBF0FBE8DBF0C
:105660001BC0CE51EC2FF0E0E057FE4F80818093BD
:105670004F0312C061E003C061E006C06AE08091A0
:105680004F030E94B82708C080914F030E945B28F7
:1056900003C089E798E013C080914F03882369F025
:1056A0001F928F9383E798E09F938F930E947407D4
:1056B0000F900F900F900F9004C080E798E00E9429
:1056C000DB0681E006C01092500380E002C080E05B
:1056D00000CFCF9108950E94722B6894B1110C9461
:1056E000012C08950E94E62B88F09F5798F0B92F5F
:1056F0009927B751B0F0E1F0660F771F881F991F07
:105700001AF0BA95C9F714C0B13091F00E94002C7C
:10571000B1E008950C94002C672F782F8827B85F8C
:1057200039F0B93FCCF3869577956795B395D9F75E
:105730003EF490958095709561957F4F8F4F9F4F68
:105740000895E89409C097FB3EF490958095709574
:1057500061957F4F8F4F9F4F9923A9F0F92F96E9BD
:10576000BB279395F695879577956795B795F11132
:10577000F8CFFAF4BB0F11F460FF1BC06F5F7F4FCF
:105780008F4F9F4F16C0882311F096E911C07723E1
:1057900021F09EE8872F762F05C0662371F096E8EA
:1057A000862F70E060E02AF09A95660F771F881FB9
:1057B000DAF7880F9695879597F9089557FD9058D1
:1057C000440F551F59F05F3F71F04795880F97FBC5
:1057D000991F61F09F3F79F087950895121613067F
:1057E0001406551FF2CF4695F1DF08C016161706AE
:1057F0001806991FF1CF86957105610508940895E3
:10580000E894BB2766277727CB0197F908950E9474
:105810001A2C0C948B2C0E947D2C38F00E94842C26
:1058200020F0952311F00C94742C0C947A2C1124F4
:105830000C94012C0E94DE2B70F3959FC1F3950F01
:1058400050E0551F629FF001729FBB27F00DB11D04
:10585000639FAA27F00DB11DAA1F649F6627B00D94
:10586000A11D661F829F2227B00DA11D621F739F7D
:10587000B00DA11D621F839FA00D611D221F749F8B
:105880003327A00D611D231F849F600D211D822FD2
:10589000762F6A2F11249F5750409AF0F1F08823F9
:1058A0004AF0EE0FFF1FBB1F661F771F881F915026
:1058B0005040A9F79E3F510580F00C94742C0C9435
:1058C000012C5F3FE4F3983ED4F386957795679576
:1058D000B795F795E7959F5FC1F7FE2B880F911D50
:1058E0009695879597F9089597F99F6780E870E0F6
:1058F00060E008959FEF80EC089500240A94161646
:10590000170618060906089500240A9412161306AD
:10591000140605060895092E0394000C11F488233B
:1059200052F0BB0F40F4BF2B11F460FF04C06F5F57
:105930007F4F8F4F9F4F0895991B79E004C0991FA7
:10594000961708F0961B881F7A95C9F780950895D9
:10595000AA1BBB1B51E107C0AA1FBB1FA617B70795
:1059600010F0A61BB70B881F991F5A95A9F78095B1
:105970009095BC01CD01089597FB072E16F4009475
:1059800007D077FD09D00E94A82C07FC05D03EF473
:10599000909581959F4F0895709561957F4F0895DB
:1059A000A1E21A2EAA1BBB1BFD010DC0AA1FBB1F23
:1059B000EE1FFF1FA217B307E407F50720F0A21B95
:1059C000B30BE40BF50B661F771F881F991F1A9402
:1059D00069F760957095809590959B01AC01BD012C
:1059E000CF010895EE0FFF1F0590F491E02D09946B
:0459F000F894FFCF59
:1059F40047094A094B094C094D094309C709AD092F
:105A040046094E090A01BD10AE118B11571123111D
:105A14000136032808140A321E524E2D3432004C2B
:105A2400554641004F4646004F4E00434F4E4E00F0
:105A3400506F776572656400556E61747461636854
:105A440065640044656661756C74004164647265E4
:105A54007373656400436F6E66696775726564008D
:105A64003F0053757370656E64656400404D362263
:105A74001906CC05960574050005190532054B0574
:0A5A840001020304050607080900EB
:10680000E70000000000000004000500060007008B
:10681000080009000A000B000C000D000E000F001C
:1068200010001100120013001400150016001700CC
:10683000180019001A001B001C001D001E001F007C
:10684000200021002200230024002500260027002C
:106850002800000035002B002C002D002E002F00FA
:1068600030002A00000033003400290036003700D1
:106870003800E00000000000000000000000000000
:106880000000000000000000000000000000000008
:1068900000000000000000000000000000000000F8
:1068A00000000000000000000000000000000000E8
:1068B00000000000000000000000000000000000D8
:1068C00000000000000000000000000000000000C8
:1068D00000000000000000000000000000000000B8
:1068E0000000000000000000310000000000000077
:1068F0000000E100E300E200F1A1E500E600000095
:106900000100010001000100EA4401000100E2442D
:106910000100010001005500460054004A004B00F0
:10692000560057004700480001000100E9440100FB
:106930000100010001000100010001003A003B00DC
:106940003C003D003E003F0040004100420043004B
:10695000580001004C00390001004400450052007D
:1069600001000100010050004F0081404D004E0029
:1069700051000100010001000100010001000100BF
:1069800001000100010001000100010001000100FF
:1069900001000100010001000100010001000100EF
:1069A00001000100010001000100010001000100DF
:1069B00001000100010001000100010001000100CF
:1069C00001000100010001000100010001000100BF
:1069D00001000100010001000100010001000100AF
:1069E0000100010001000100490001000100010057
:1069F000010001000100010001000100010001008F
:00000001FF
